:10100000509F0600F209F209D60AD60AD208D10882
:1010100024FF7821FFFFFFFFFFFFFFFFFFFFFFFF20
:1010200035200000008E2001BB00000003003DB20F
:10103000CA5800000000000000000000000000008E
:1010400000000000000000000000000000000000A0
:10105000008E268E2101FFFFFFFFFFFFFFFFFFFF36
:10106000FFFFFFFFFFFFFFFFFFFFFFFFFFFFFFFF90
:10107000FFFFFF0070820952FF0000000000000027
:101080002B4C021A740802000000E803E803000079
:10109000E4070000FFFFFFFF00FFFFFFFFFFFFFF70
:1010A000FFFFFFFFFFFFFFFFFFFFFFFFFFFFFFFF50
:1010B000FFFFFFFFFFFFFFFFFFFFFFFFFFFFFFFF40
:1010C000C085FE16FFFFFFFFFFFFFFFFFFFFFFFFD3
:1010D000FFFFFFFFFFFFFFFFFFFF08100080000082
:1010E00046808F0BBF0DA780EE063C08FE08FFFF71
:1010F000FFFFFFFFFFFF0108998F9D8E8C8D3D87BD
:10E00000314000063C4066033D400801B012AEFCC2
:10E01000B012B0F1B012DAFC32C23140FE0532D299
:10E02000F240F30001033E4080100F43FF4E020315
:10E030001F533F900A00FA23F2400B0000033540C3
:10E040000003B0125CE9F240E1005004F24003002A
:10E050005104B01214E7B012ACECF24005005E04BB
:10E06000B0121EFCF2B003005D04212CF2401E0031
:10E070005404B2B010006201CB29C2935404F923B6
:10E08000D2835E04ED23F240F1000103D243020388
:10E09000E243000335400003B0125CE9F2400600A1
:10E0A0005404C2935404FD2382432001FD3FC24324
:10E0B0005F04C243600482436C03B012FEE1F2903D
:10E0C000050066043034B2B010006201A129B2B07C
:10E0D000100064017E28D2B30100F12FF240AF009E
:10E0E0000604D2535F043E400604D2425A040003A1
:10E0F000B01220E2B012FEE1B01294E482436C034D
:10E10000F290030008040524D2436604C24361046C
:10E11000D63FF290030061040334D2536104CF3F31
:10E12000E2436604CC3FF240F40001033E4080101D
:10E130000F43FF4E02031F533F900A00FA23F240A1
:10E140000B00000335400003B0125CE9D2C3190094
:10E15000E2C32900C2436004C2435F0482436C03EC
:10E16000F2402700010338400103D2435904B012A2
:10E17000A8E7B01210E2F2401E005404C293540407
:10E180009E27D2B30100FA2FB01286F93E40060452
:10E19000F24031000003B01220E2B012FEE1B012F2
:10E1A00094E48D3FF2409F000103F24023000203FC
:10E1B000D2424C04000382436C03D2536004B01279
:10E1C00030E2D2424C04000335400003B0125CE957
:10E1D000763FB01284F7733F3FF03F003F50A00FEF
:10E1E00012C30F10F0400700A821C04FA3213F40E9
:10E1F00010002B433C408F03B0121CE8D33DF2408B
:10E200008F005B04F24020005C04B01284E73041D0
:10E21000F24047005B04C2435C04B01284E7304123
:10E220000F43FF4E01031F535F920003FA23304157
:10E23000B012A8E4B01270ECA2C36001D24276031F
:10E240003F03D24277034003F2D080004003F2D074
:10E2500020004003D24255043E030E435E42550463
:10E26000A2D360010E5E0E5ED24E041041031E5317
:10E27000D24E041042031E53D24E041043031E53C9
:10E28000D24E04104403B012E2EAB01228EBB012EE
:10E2900036EBC24E48038E10C24E4903B01294EAC8
:10E2A000B01228EBB01236EB0E110E11C24E450320
:10E2B0008E10C24E4603B01248EAB01228EBB012DC
:10E2C00036EB0E110E110E110E11C24E4703B01295
:10E2D000AEEAB01228EBB01236EBC24E4C038E10F1
:10E2E000C24E4D03B01230EAB01228EBB01236EB3A
:10E2F000C24E55038E10C24E5603B01218EAB01229
:10E3000028EBB01236EBC24E57038E10C24E5803A4
:10E31000B01262EAB01228EBB01236EBC24E4E03D6
:10E320008E10C24E4F03B0127CEAB01228EBB0122E
:10E3300036EBC24E59038E10C24E5A03A2C360017F
:10E34000C2435704D2435804A2D36001B2900F00D5
:10E350006C031B2CB2B010008401F82FB2900E0099
:10E3600072032634B2900D0072030520B29021DFB3
:10E3700070031E34003CD24270033503D242710355
:10E380003603D24272033703213CB2B0100084013D
:10E390001928B2C01000840182936E030920B24391
:10E3A0007003B240FF007203B2C010008401E33F6B
:10E3B000B24021DF7003B2400D007203B2C0100002
:10E3C0008401D93FB2C010008401D53FD240A62CB1
:10E3D0003203D240A12C3303D2409C2C3403D240D0
:10E3E000982C3803D240932C3903D2408B2C3A031B
:10E3F000D0408E2C6C1FD040892C671FD040842CBD
:10E400005D1FD040802C591FD040792C521F3041C5
:10E41000D2424E044D04B012C0FCF2D08000580429
:10E42000D2C30100E2C31900F2C020003300F2C0E1
:10E4300020003200D2C31F00D2C31E00F2C0200051
:10E440002A00F2C22A00F2C010002A00F240E100C5
:10E450005004C2435104B01214E7F2900500660460
:10E460003634B2B010006201F82FF29003008B0333
:10E47000CF27F29062008B032E24F29061008B0371
:10E480005024F29060008B037A24F29057008B03A3
:10E490008924C33FB01230E2D2424C04000335401D
:10E4A0000003B0125CE93041A2D36001034303438F
:10E4B0000343034303430343A2C36001A2B3A00188
:10E4C000F32FF2D080005804A2D360013041D2C3B0
:10E4D0001900E2C329000B430C430F435B428E0338
:10E4E0004B939B273B902100982F5F428D033F90D9
:10E4F0008000932F0C4F0C5B3C9081008E2F3C4092
:10E500008F03F2900A008C030824F2900B008C0316
:10E510008423B01228E8053C803FB0121CE8013C7F
:10E520007C3F0B430C430F435B428E034B93752799
:10E530003B908100722F5F428D033F9080006D2FD2
:10E540000C4F0C5B3C908100682FF2900A008C030A
:10E550000724F2900B008C0360233D400410023C22
:10E560003D4080100D5FB012CCFCF24005004D0420
:10E57000B0120EFBB012C8E6B0126AFC4E3FD24396
:10E580005804B01230E2B012CCFCE2434D04B01299
:10E590000EFB3D4032037B403100B012C8E6B012A2
:10E5A0006AFC3B3FD2D30100F2D020003300F2D00E
:10E5B00020003200D2D31F00D2D31E00F2D02000A0
:10E5C0002A00F2D22A00F2D010002A00E2D3190069
:10E5D000B240B4DC860382438803B01252FCD243BB
:10E5E00058043B41B01208FA3B4010000E6EB012C6
:10E5F00006E61B83FB233B4010000C6CB01206E6C2
:10E600001B83FB23273C0428F2D010002900033C85
:10E61000F2C01000290003430343034303430343B1
:10E620000343F2D020002900034303430343034381
:10E6300003430343034303430343034303430343AA
:10E64000F2C0200029000343034303430343034371
:10E65000034330410343034303430343034303435F
:10E66000F2D2290003430343034303430343034319
:10E67000034303430343034303430343F2C2290019
:10E680000343034303430343034303433041F2C0C3
:10E6900020002900F2C229003E4044031C40742996
:10E6A000B012E8E51C40D21E1E40D01EB012E8E5B4
:10E6B0000E433C40E25FB012E8E53E4074003C404F
:10E6C000AF18B012E8E530410C43F04D9A1CF090C1
:10E6D0001000941C0520B012ECE6F0401000881CDD
:10E6E000B012ECE61C530B9CF0233041D243530490
:10E6F000B2400900680312127001B150A00100007D
:10E70000B2417201B240B0006201B2B010006201C9
:10E71000FC233041C2434E04D2C34F04E2C34F0432
:10E7200082436A03C2435304B24009006803B24003
:10E73000149162013041D2C30100F240D000620066
:10E74000C2436300F24006006400F2D030001B00B8
:10E75000C2436000F240800061003041D2C301003A
:10E76000F24082006200F24006006300F2400600C0
:10E770006400F2D030001B00C2436000F240800011
:10E7800061003041D2C30100C2435D04C243650051
:10E790008043DB1CD2D301003041E2B30300FD2BE8
:10E7A000D240D61B67003041F0401000CC1BB012A5
:10E7B0009AE7F890100000000520F0401000BA1B06
:10E7C000B0129AE7F048B21BB0129AE7D0838B1CC4
:10E7D000F023F0401000A21BB0129AE7F0400300B3
:10E7E000981BB0129AE730413F4010002B433C4049
:10E7F0008F03B0121CE830413F400E001B433C40E9
:10E800008F03B0121CE830413F400F001B43D2433E
:10E810008F033C408F03B0121CE830413F90400012
:10E8200009343D4080100F3C3F90400008343D408B
:10E830000410093C3F8040003D404010043C3F80B4
:10E8400040003D40401032C20D12B01268E82D4128
:10E85000B012A6E8FF4CC6031F531B83FB233D41A8
:10E86000B0127AE832D230410E43AE4DC6032D537A
:10E870002E533E904000F9233041B04000A5AE1821
:10E88000B04040A5A4180E439D4EC60300002D5372
:10E890002E533E904000F823B04000A58C18B040A5
:10E8A00010A58A183041B24000A52C0192B32C016A
:10E8B000FD2FB24002A52801CD43000092B32C01E8
:10E8C000FD2FB24010A52C01304105120B430E4321
:10E8D0005E4200035E830D437D453F421DB3013C14
:10E8E0004D6D0C6C0B120B100CEB0B100B100CEB9A
:10E8F0000B100B100CEB2B410B6B0B6B0B6B0CEB26
:10E900003B410C100B6B1F83EB231E83E42335412B
:10E910003041D24229042804D2422B042904D24295
:10E920002D042A04D2422F042B04D24231042C0499
:10E93000D24233042D04D24235042E04D24237048D
:10E940002F04D24239043004D2423B043104D24273
:10E950003D043204F2409F0006043041F2C08000C2
:10E960006203D2536203F290650062030228D2432D
:10E970006203B2D0800062030F3CD2924C040003C9
:10E980000B24F290470001030720D25300035F429B
:10E990000003DF4262030103D2D31F00F2D08000E4
:10E9A0002900B0128CECE2435404C2935404FD23BA
:10E9B000E2530003B012CAE80F435F420003CF4B9B
:10E9C00000031F838B10CF4B0003D24200034D0482
:10E9D0005B420003F24080006204B04010009C19CA
:10E9E0000D451D53B012CCFCF040E2007A19B01274
:10E9F000ECE6F04055007019B012ECE6D0424D0440
:10EA00006619B012ECE6B012C8E6B0126AFCB0901B
:10EA100022006819FC233041A2C3A0018243A40153
:10EA20004D43B240F00FA001B240F202A201663C99
:10EA3000A2C3A0018243A4015D43B240F00FA00134
:10EA4000B240F202A2015A3CA2C3A0018243A40137
:10EA50007D401200B240F00FA001B240F202A201CC
:10EA60004D3CA2C3A0018243A4017D400300B240FB
:10EA7000F00FA001B240F202A201403CA2C3A001EB
:10EA80008243A4016D42B240F00FA001B240F202F5
:10EA9000A201343CA2C3A0018243A4017D40150021
:10EAA000B240F00FA001B240F202A201273CA2C383
:10EAB000A0018243A4017D401600B240F00FA001E6
:10EAC000B240F202A2011A3CA2C3A0018243A401F7
:10EAD0007D400700B240F00FA001B240F202A20157
:10EAE0000D3CA2C3A0018243A4017D401A00B240A4
:10EAF000B00FA001B240F202A201003CC24D800062
:10EB0000C24D8100C24D8200C24D8300C24D8400BF
:10EB10007DD08000C24D8500034303430343A2D34D
:10EB2000A00192D3A0013041B2B02000A401FC2B7F
:10EB3000A2C3A00130413F4040010E4F0D4F2F5363
:10EB40002C4F2C9E01380E4F2C9D01340D4F3F90C1
:10EB50004A01F5230E9D01202E538E4300008D4364
:10EB600000003F4040012E4F2F532E5F3F904A013F
:10EB7000FB230E110E113041331291830000FD234F
:10EB800021533041B240805A2001E2D32200E2D327
:10EB90002600F0C018008B14F0D0E0008514E2D2FB
:10EBA0002600E2D22E00F240BA002A00F2C0200075
:10EBB0002900F2C22900F2D010002900E2C3290086
:10EBC000D2D31A00E2D21A00E2D31A00D2C319003B
:10EBD000E2C21900E2C31900F24009001E00D2D3BC
:10EBE0001F00E2D31F00F2D020003200F2D020003C
:10EBF0003300F2D040003200F2D040003100F2D0B9
:10EC000080003200F2C080003100F2C23300F2D244
:10EC10003200F2C23100F24337003041F2C08000CE
:10EC20005700F2D080005300F2D020005300E2C31E
:10EC300002003F40FF471F83FE23E2B30200F72399
:10EC4000B01278EBF240880058003041A2426201D5
:10EC5000B24024006201B24062026001304182434E
:10EC60006C03B24046028001B2D0200080013041E6
:10EC700032C282436C038243700382437203824335
:10EC80006E03B2401041840132D2304182436C03A2
:10EC900012129001B15040030000B2419201B04005
:10ECA0002200D816B240900082013041C243630472
:10ECB000B042CA16B240308164013041F24562046C
:10ECC000A053B816B0F00F00B2160B20C293000389
:10ECD0000620F2420003B0402400A016023CD2837A
:10ECE0000003D25262046204182CB2504003920115
:10ECF0003041B25040039201D28300030D20B04056
:10ED000022007816B2C010008201F2C080002900F3
:10ED1000D2C31F00D2C31D003041B250A0019201E6
:10ED200090D358163041B250A001920190C34C16B6
:10ED30003041B0F01F0044160224A0533E16D252B8
:10ED400062046204EA2FB250400392013041B25093
:10ED5000A0019201A0532416304110521E013041EF
:10ED6000083C3041304130413041304192536C03D6
:10ED70003041A2B384010B28B2C010008401A2C3A9
:10ED8000840182437203B2400F00700330418293CA
:10ED90006E03092092429401700392426C03720345
:10EDA00092536E0330419290E2226E032338B2C038
:10EDB00010008401A2C3840112126C0391827203B9
:10EDC0000000B241720392B3800182637203082093
:10EDD00012129401918270030000B241700330411D
:10EDE00092837203B2E370039252940170038263C0
:10EDF000720330418293940192536E0330410A12A0
:10EE00000B120D120C120F120E1210522E01C93DD0
:10EE1000043CC73DC63DC53D403C32C0D000925287
:10EE20007E037401B2B000106401162882937C0343
:10EE30000420B2C010006401B43DB2D0800064016F
:10EE4000D2B363040328B2C08000640112C352101D
:10EE50006304B2537C03A53DB2B0000164010A28EB
:10EE6000B2C0000164011E427E0312C30E10825E16
:10EE70007401973D12C352106304B2B000046401E0
:10EE80000328F2D080006304B2537C0382937C0396
:10EE90008821B2C010006401843DF2905C006704D8
:10EEA000032CD2536704023CC24367045E426604EB
:10EEB0004E8338245E8307245E8366245E83192490
:10EEC0005E833024763C5E4267045E8307247E8046
:10EED0001E0008247E803C0009246B3CF2D0800098
:10EEE0003100673CF2C080003100633CC2436704DC
:10EEF000603C5E4267045E830A245E830C245E836A
:10EF000006245E8308247E801B000924523CF2D034
:10EF1000800031004E3CF2C0800031004A3CC243C8
:10EF20006704473CB290C1117E0316205E4267041D
:10EF30005E8305246E8207246E8209243A3CF2D057
:10EF400080003100363CF2C080003100323CC243C8
:10EF50006704D25368042D3C5E4267045E83072435
:10EF60007E801E0008247E801E000924223CF2D0F0
:10EF7000800031001E3CF2C0800031001A3CC243C8
:10EF80006704D2536804153C5E4267045E8307241D
:10EF90007E80050008247E80190009240A3CF2D0F6
:10EFA00080003100063CF2C080003100023CC243C8
:10EFB0006704C29366042F24D2B32800142CD29382
:10EFC00068040428F2D080003100253CE242660447
:10EFD000B290C1117E031F20F2900A0067041B2823
:10EFE000C2436704183CD29368040428F240050029
:10EFF0006604113CC29368040E24C2436804C243F1
:10F000006704B290C1117E030420F240030066043D
:10F01000023CD2436604C29354040224F2535404C3
:10F02000C29365040324F2536504023CC2436404A2
:10F03000C2935804B638C29356040520D2435604EE
:10F04000B0122EFAAE3CC29358048320B2B0200016
:10F05000A401A728A2C3A0014D433C40FF0F4F438A
:10F060007F9006000C2C4E4F0E5E1C9E4001052822
:10F070004B4F0B5B1C4B40014D4F5F53F13F4B4DD2
:10F080000B5B8B4340014D430C434F437F90060085
:10F090000C2C4B4F0B5B1C9B4001052C4B4F0B5B0F
:10F0A0001C4B40014D4F5F53F13F4B4D0B5B8B436E
:10F0B0004001824376034F437F900600072C4B4F5D
:10F0C0000B5B925B400176035F53F63F12C3121055
:10F0D000760312117603D242560457045E42560458
:10F0E0005E8305245E8307245E830A240D3C0C4363
:10F0F0003A40B80B093C3C4078053A401C0C043CB3
:10F100003C4020033A40FF0F829C7603082CE29398
:10F1100056041028F2535604B0122EFA0B3C1A92E1
:10F120007603082CF29003005604042CD2535604A4
:10F13000B0122EFAD24358045E4257047E53C24E98
:10F140005504F290030056042C20F2D0800058049D
:10F15000283CF2535804C29358042320A2C3A001B0
:10F160008243A401B240F00FA001B240F202A2011A
:10F17000F24007008000F24007008100F2400700E3
:10F180008200F24007008300F24007008400F24052
:10F1900087008500034303430343A2D3A00192D316
:10F1A000A0013E413F413C413D413B413A410013BA
:10F1B000B2B040002C010328B24040A52C01C2434C
:10F1C0000003C2430103C2433203C2433303C243B9
:10F1D0003403C2433503C2433603C2433703C24339
:10F1E0003803C2433903C2433A03D24210103B03EF
:10F1F000C2433C03C2433D03C2433E03C2433F03F9
:10F20000C2434003C2434103C2434203C2434303D8
:10F21000C2434403C2434503C2434603C2434703B8
:10F22000C2434803C2434903D2428F104A03D24229
:10F2300098104B03C2434C03C2434D03C2434E03D9
:10F24000C2434F03F29224100320D2435003023CE6
:10F25000C2435003C2435103C2435203C243530348
:10F26000C2435403C2435503C2435603C243570328
:10F27000C2435803C2435903C2435A03F2435B03D8
:10F28000D2428E105C03C2435D03C2435E03C2439D
:10F290005F03C2436003C2436103C2436203C243CC
:10F2A0006303F24062004C04C243C60382436C0312
:10F2B00082436E038243700382437203824374036A
:10F2C000C2435904C2435E04C2435F04C2436004A4
:10F2D000C2436104C24362048243820382438403C3
:10F2E000C2436904C2436A0432C20343F24080004D
:10F2F0005804C2434E04C2434F04B01284EBB240E0
:10F300000C8E7E03B0121CECB0124CECB0125EEC12
:10F31000B01298FCB012ACEC32D2C2436604D243B5
:10F320006804C29373101A20E2B21C00172CD2D3C7
:10F3300019003E40204E0F430D4E0DDF0D93032468
:10F340003E533F63F93FE2D21900E2D31900F2D0F5
:10F3500080003100D2436604B01208FAD2D31900FB
:10F36000E2C21900E2C31900D2B32800FD2BD293E8
:10F3700068040E28F2D080003100E2D21900E2D3F6
:10F380001900C2436804D2436604B01208FA023C72
:10F39000D2C319001C4330410F12B250A0017201B8
:10F3A000C29353042324929368030620B2C08000C2
:10F3B0006201B2536803BD3C829368030720B2C068
:10F3C00010006201B2C080006201B33C92B36603D8
:10F3D0000428B2C080006201033CB2D08000620108
:10F3E00012C312106603B2536803A33CB290090023
:10F3F00068030920B2C000016201B250D00072015E
:10F40000B2536803963C829368031424B2B000049C
:10F4100062010428B2D080006603033CB2C08000C1
:10F42000660392936803032412C312106603B25357
:10F4300068037F3CB2D014816201B24009006803C6
:10F4400082936A031F201F4266033F8003000C243F
:10F450003F800D000F20C29352040324C243520484
:10F46000683CD2435204653CC29352046224C243B6
:10F4700052045F3CD24266038A0392436A03C2434A
:10F480005204573CB29063006A03512C1F4266033A
:10F490003F80030013243F800D003F20C29352049D
:10F4A0000A24C24352041F426A03DF4266038A03EE
:10F4B00092536A033E3CD24352043B3CC2935204F3
:10F4C0002424C2435204D2426A034E04C29350041D
:10F4D0001924D2928A0350041520C29351040420A7
:10F4E000B2C010006201253CC29351040824D2929C
:10F4F0008B0351040420B2C0100062011A3C824305
:10F500006A03173C82436A03143C1F426A03DF42CA
:10F5100066038A0392536A030C3CC24352041F429F
:10F520006A03DF4266038A0392536A03023C824302
:10F530006A033F4100130A124A4C4E4A4E83032489
:10F540006E835724AB3CB24024007803B0129AE794
:10F55000B24050007803B0129AE7B2404D007803F1
:10F56000B0129AE7B24054007803B0129AE7B24062
:10F570004B007803B0129AE7B24033007803B01220
:10F580009AE7B24035007803B0129AE7B2403300F0
:10F590007803B0129AE7B2402C007803B0129AE7D1
:10F5A000B24031007803B0129AE7B2402C007803E1
:10F5B000B0129AE7B24030007803B0129AE7B24036
:10F5C0002A007803B0129AE7B24033007803B012F1
:10F5D0009AE7B24036007803B0129AE7B2400D00C5
:10F5E0007803B0129AE7B2400A007803B0129AE7A3
:10F5F000553CB24024007803B0129AE7B240500064
:10F600007803B0129AE7B2404D007803B0129AE73F
:10F61000B24054007803B0129AE7B2404B0078032E
:10F62000B0129AE7B24033007803B0129AE7B240C2
:10F6300035007803B0129AE7B24033007803B01275
:10F640009AE7B2402C007803B0129AE7B24031003A
:10F650007803B0129AE7B2402C007803B0129AE710
:10F66000B24031007803B0129AE7B2402A00780322
:10F67000B0129AE7B24033007803B0129AE7B24072
:10F6800037007803B0129AE7B2400D007803B01249
:10F690009AE7B2400A007803B0129AE73C40D007DC
:10F6A0000D43B012C8FA3A413041E2C21900E2C338
:10F6B0001900F2F003002200F2C020002900F2C27B
:10F6C0002900F2C010002900F2C080002900F2C019
:10F6D00010001B00F2C010001900F2C0200033001F
:10F6E000F2C020003100F2C040003100E2D3290016
:10F6F000D2C31900B012ACECF24003006604C2435E
:10F700006704D242FE105600D242FF105700C24397
:10F710005800F24020005300B240C1117E03F2C0F5
:10F7200080003100F290050066040520D2C3190064
:10F73000E2C32900FF3FB2B010006401F32FB01202
:10F7400084F74C93EF27B01284EBD2435604B012E7
:10F750002EFAF2D010001B00D2D319003E40204EEA
:10F760000F430D4E0DDF0D9303243E533F63F93FCE
:10F77000E2D31900E2D21900E2C32900B012E4FB7F
:10F78000304008FA0A124A43C29363045824C24321
:10F7900064045E4263047E80410007247E800C0086
:10F7A00007247E8005000624083CB012AAF6473CD8
:10F7B0005A43453CB01208FA423CF290810063047F
:10F7C0003128F290BD0063042D2CF29003006604F2
:10F7D0002320B01284EBD2435604B0122EFAF2D09A
:10F7E00010001B00F2D020003300D2D31900E2C376
:10F7F00029003E40A0861F430D4E0DDF0D930324CC
:10F800003E533F63F93FE2D21900E2D31900B01230
:10F810001CECB2400C8E7E035C426304B0124AFBC7
:10F820005A430D3CF290200063040928F2903F00F7
:10F830006304052C5C426304B01238FC5A43B012D6
:10F84000ACEC4C4A3A4130410F12E2B26500042858
:10F85000F2F083006500483CF290AA0066001F2089
:10F86000E2936B040D20C2436B04D2436C045F42ED
:10F870006D044F4FDF4266000604D2536D04343CE2
:10F88000C2936C0409245F426D044F4FDF4266004F
:10F890000604D2536D04283CD2536B04253CC2931A
:10F8A0006C042024F2903C006D0413285F426D0428
:10F8B0004F4FDF4266000604D2536D04C2436C040E
:10F8C000D2426D045A04F24027005A04D2C3010008
:10F8D0000B3C5F426D044F4FDF4266000604D2537B
:10F8E0006D04023CC2436B043F4100130D120C1225
:10F8F0000F120E1292B37A030328B01226ED3E3C8B
:10F900001F427A033F902500392C0F5F104F10F9EA
:10F910005AF97CF960F97CF960F97CF960F97CF9B5
:10F9200060F97CF960F97CF960F97CF960F97CF99F
:10F9300066F97CF96CF97CF966F97CF966F97CF971
:10F9400066F97CF96CF97CF966F97CF966F97CF961
:10F9500066F97CF972F97CF978F9B012BCEC0E3CCE
:10F96000B012C0EC0B3CB01232ED083CB0124EEDC0
:10F97000053CB012EAEC023CB012F2EC3E413F41D1
:10F980003C413D4100130A122182F2404900060425
:10F990004A437A900C00352C4F4A0E4F0F5F0F5F91
:10F9A0000F5E4E4A0E5EDE4F080408044F4A0E4FAB
:10F9B0000F5F0F5F0F5ED14F0C0400004F4A0E4FD8
:10F9C0000F5F0F5F0F5ED14F0B0401004F4A0E4FC8
:10F9D0000F5F0F5F0F5ED14F0A0402004F4A0E4FB8
:10F9E0000F5F0F5F0F5ED14F090403002C411D41D3
:10F9F0000200B012B2FB4F4A0F5FCF4C09045A53BA
:10FA0000C83F21523A413041B01218FDB0128EE683
:10FA1000D2B32000FD2BD2428E105C03D2428F1055
:10FA20004A03D24210103B0332D2304018E05E420B
:10FA300056045E8305245E830C245E8313241A3CE3
:10FA40005E4222007EF003007ED08000C24E220083
:10FA5000113C5E4222007EF003007ED05000C24E78
:10FA60002200083C5E4222007EF003007ED0280087
:10FA7000C24E2200F240050058043041061207121F
:10FA8000064D7DD0800006660767861076F3768087
:10FA90007F001428768018000A28369212340C5CF5
:10FAA0000D6D5683FC2F071037413641304176E308
:10FAB000FA270D110C105683FC23F53F0C430D4320
:10FAC000F23F3C433D43EF3F12C30D100C100212B6
:10FAD00032C20343824C3001B240D00738011C428D
:10FAE0003A0192423C013A01824D3401B240D007C2
:10FAF00038011D423A0132410E430F430F9D032846
:10FB000005200E9C032C1E530F63F83F30410A1250
:10FB1000F240E2008A030A43C2934D041424FA908F
:10FB200010008A030520B24010006603B012ECE614
:10FB30005F4A8A034F4F824F6603B012ECE6F253DE
:10FB40004D041A53E93F3A4130410A1221834A4C8D
:10FB50004C4A3C50200F2E43B01282FB814C0000D7
:10FB6000D24101009003E2418F03B012E8E7B012E6
:10FB700008FA4C43B01236F521533A4130418C110A
:10FB80008E11091209430E9303343EE31E5319D319
:10FB90000C9303343CE31C5339E3B01206FC19B355
:10FBA00002243CE31C5329B302243EE31E53394193
:10FBB0003041B0127CFA0F283D90008006200C9353
:10FBC00009243D4000800C433041FB2F3CE33DE3E2
:10FBD0001C530D6330413DB00080FC273D40FF7F4A
:10FBE0003C433041D2436604D2D31900E2C329001A
:10FBF000E2D21900E2D31900B2400C8E7E033040ED
:10FC00001CEC7CF37EF30F4E0D4C0E431C430D5D3C
:10FC10000E6E0E9F01280E8F0C6CF92B3041B01226
:10FC200036E7F2D003005D043C40D0070D43B0122C
:10FC3000C8FA4C43304036F50A124A4C4E4A7E50C0
:10FC4000E000C24E8F03B012F8E7B01208FA3A4152
:10FC500030411E4286031F4288030D4E0DDF0D9377
:10FC600003243E533F63F93F3041B2401000660326
:10FC7000B012ECE6B24003006603B012ECE630408E
:10FC800014E70D120C120F120E12B0125AED3E4173
:10FC90003F413C413D410013C2435504824376033A
:10FCA000C2435604C2435704D243580430410F4C58
:10FCB0000F5D033CCC4300001C530C9FFB233041E1
:10FCC000B012CCFCB0120EFB30406AFCB240100007
:10FCD00066033040ECE63040DEFC3040D6FCFF3FAF
:10FCE00009120A120B120A430B43394020000C5C24
:10FCF0000D6D0A6A0B6B0A8E0B7F04281CD33953D7
:10FD0000F623043C0A5E0B6F3953F1230E4A0F4B66
:10FD10003B413A41394130415C4200108C101D4258
:10FD200002108D105A4201100DEA0F433E40F401BB
:10FD3000B012E0FC0C5C0D6D0C5C0D6D1C53804C26
:0CFD40003808804D36083041FFFFFFFFFF
:10FFE000FFFFFFFFFFFFFFFFFFFFFFFFFFFF48F8DF
:10FFF000FEED98F3FFFFFFFF82FCECF8FFFF00E04F
:00000001FF
